:1000000015C100002EC100002CC100002AC1000053
:1000100028C1000026C1000024C1000022C1000048
:1000200020C100001EC100004CC20000C4C200007C
:1000300018C1000016C1000014C1000012C1000068
:1000400010C100000EC100000CC100000AC1000078
:1000500008C1000006C1000004C1000087C1000003
:1000600000C10000FEC00000FCC00000FAC000009B
:10007000F8C00000F6C00000F4C00000F2C00000AC
:10008000F0C00000EEC00000ECC00000EAC00000BC
:10009000E8C00000E6C00000E4C00000E2C00000CC
:1000A000E0C00000DEC00000DCC000000001000075
:1000B0000C02120002000086014900220000F0013B
:1000C0001C0021000098010900220100CF0121003D
:1000D000210100B8010900030000820104010309A5
:1000E000044C01340203090424012603030904F229
:1000F0000030300345006D0075006C006100740035
:100100006500640020004100720064007500690011
:100110006E006F00200053006500720069006100EE
:100120006C00000026035400650065006E0073003B
:1001300079006400750069006E006F0020005200B5
:100140006100770048004900440000003403540077
:10015000650065006E007300790064007500690039
:100160006E006F00200052006100770048004900D7
:1001700044002000440065007600690063006500CB
:1001800000000403090409024900020100C0320909
:100190000400000203000002092111010001221CD9
:1001A000000705830340000107050403400001091F
:1001B00004010002030000030921110100012221B2
:1001C0000007058103400001070502032000020625
:1001D000C9FF0904A15C7508150026FF00954009B8
:1001E00075810295200976910295040976B102C0C5
:1001F00006ABFF0A0002A1017508150026FF009555
:100200004009018102954009029102C012010002D9
:1002100000000040C016860402010001000101C177
:100220003601C02601C13601C036000011241FBEB0
:10023000CFEFDAE0DEBFCDBF11E0A0E0B1E0ECE14E
:10024000F9E002C005900D92A030B107D9F721E086
:10025000A0E0B1E001C01D92A930B207E1F758D388
:100260005BC3CECE569A08955E9A68EE73E080E046
:1002700090E0BCD05E9868EE73E080E090E0B6C09D
:100280001DBA109268001CBC10BE1FBA10927A00F2
:1002900010926E0010926F00109271001092720016
:1002A0001092C900ECEBF0E0108214B817B81AB83D
:1002B0001DB810BA108215B818B81BB81EB811BAFC
:1002C0000895F894E1E6F0E020E8208381E080835F
:1002D00093E094BD95BDEEE6F0E09081916090834F
:1002E0008093800092E0909381008093900090939F
:1002F00091009093C00094E09093C1008093C2005D
:100300008093C3001092C40085E880937A00209304
:100310007B0010927E0010927D00A9D07894089501
:10032000F89484B7877F84BF809160008061809358
:1003300060001092600080E197E20197F1F781E0A0
:100340008093E00080E28093D80080E395E70197F6
:10035000F1F796DF0C94003FFFCFF89491DF80E334
:1003600095E70197F1F70C940000FFCF8F938FB7BB
:100370008F93809100018A5F8D37D0F480930001C4
:10038000809101018E5F80930101D8F0809102017C
:100390008F4F80930201A8F0809103018F4F8093CB
:1003A000030178F0809104018F4F8093040109C00C
:1003B0008D5780930001809101018D5F8093010131
:1003C00028F780910501885F8093050158F080919E
:1003D00006018F4F8093060128F0809107018F4F0F
:1003E000809307018F918FBF8F911895CF92DF92E5
:1003F000EF92FF926B017C0119D09B01C114D104D3
:10040000E104F10429F4FF90EF90DF90CF9008957C
:100410000DD0621B730B683E734080F381E0C81AF5
:10042000D108E108F10828513C4FE8CF0FB6F89405
:1004300066B515B270910501809106019091070192
:100440000FBE10FE05C06F3F19F0785F8F4F9F4FB2
:1004500011240024660F001C660F001C660F001C90
:10046000702908958091E80080FFFCCF0895809165
:10047000D80087FF02C085FF23C081E08093D700AA
:1004800080EA8093D80082E189BD09B400FEFDCFE7
:1004900080E98093D8001092E00010920F01109232
:1004A0000E0110920D0110920C0110920B0110928E
:1004B0000A01109209011092E1008CE08093E200A1
:1004C00008951F920F920FB60F9211242F938F93BE
:1004D0009F932091E1001092E10023FF0FC0109242
:1004E000E90081E08093EB001092EC0082E38093BE
:1004F000ED0088E08093F00010920F0122FF2FC0E2
:1005000080910F01882359F180910D01882379F0A2
:10051000815080930D0181110AC081E08093E90030
:100520008091E80085FD44C08AE38093E8008091D3
:100530000B0190910C01882331F0815090E0909351
:100540000C0180930B018091090190910A0188238D
:1005500031F0815090E090930A018093090120FFCF
:100560000CC080E18093E20010920F0181E0809343
:100570000E0180EA8093D80019BC80910E01882377
:1005800079F024FF0DC082E189BD09B400FEFDCFE2
:1005900080E98093D8008DE08093E20010920E01F4
:1005A0009F918F912F910F900FBE0F901F901895D4
:1005B0001092F100B5CF1F920F920FB60F92112437
:1005C000EF92FF920F931F932F933F934F935F935D
:1005D0006F937F938F939F93AF93BF93CF93DF934B
:1005E000EF93FF931092E9008091E80083FF21C010
:1005F000E090F100F090F100C091F100D091F10095
:100600000091F1001091F1002091F1003091F10082
:1006100082EF8093E80086E0F8125AC08AE0ECEAA4
:10062000F0E045915591C417D50739F035968150C2
:10063000C1F781E28093EB002BC0459155910417DF
:10064000150711F03396F3CF4591559184912F3FC3
:10065000310519F010F02FEF30E0821708F4282F41
:100660003EEF8091E800982F9570D9F382FD10C07D
:10067000822F213408F080E4982F911122C0922F0C
:10068000981B892F3093E800911119C02034B8F4D9
:10069000FF91EF91DF91CF91BF91AF919F918F919A
:1006A0007F916F915F914F913F912F911F910F918A
:1006B000FF90EF900F900FBE0F901F901895282F6E
:1006C000D0CFFA0145914093F100AF019150D5CFC1
:1006D00085E0F81208C08EEF8093E800C3DEC068A2
:1006E000C093E300D5CF99E0F91222C0E11067C0B2
:1006F000C0930F0110920D018EEF8093E80081E00E
:10070000EEE1F2E08093E90095919093EB0099235C
:1007100031F095919093EC0095919093ED008F5F5F
:10072000853081F78EE18093EA001092EA00B0CF25
:1007300088E0F8120CC090E8E91241C093DE809185
:100740000F018093F1008EEF8093E800A1CFF110AC
:1007500012C088DE22E8E21209C00093E900F0909E
:10076000EB00F5FAFF24F0F81092E900F092F100A6
:100770001092F100E8CF8F2D8D7F813001F582E05E
:10078000E8121DC0209709F09BC0402F4F778FEFD4
:10079000840F853008F094C08EEF8093E80040937A
:1007A000E90093E0F91609F444CF89E18093EB0066
:1007B00081E090E001C0880F4A95EAF7B4CF0115B7
:1007C000110509F081C021EAE21223C081E0F8128C
:1007D00030CF80E43EEF01C0892F9091E800292FAF
:1007E0002570D9F392FD54CF982F813408F090E40E
:1007F000292F21110AC0282F291B922F3093E8009E
:100800002111EACF803440F743CF1092F1002150FC
:10081000F0CF81E2E81249C099E0F9120ACF809145
:10082000E80082FFFCCF8BEF8093E8001BDE8BCFCC
:100830001092F10091505EC089E0F81236C091E24A
:10084000E912F7CEC115D34009F0F3CE24303105BB
:1008500009F0EFCE8091E80082FFFCCF3091F100EB
:100860002091F1009091F1008091F1004BEF4093C5
:10087000E8004EEF4093E800393A51F4253409F08E
:10088000D8CE923C09F0D5CE8B3609F0D2CE48DDD9
:100890003B3809F0CECE253C09F0CBCE9D3109F096
:1008A000C8CE803709F0C5CE58DD99ECF912C1CE1B
:1008B00020E4E212BECE8EEF8093E800D3DDF4CFC9
:1008C0000115110509F4B5CE0130110571F781E06C
:1008D000F812B2CF91EA3EEFE912ABCE8091E80078
:1008E000982F9570D9F382FDD3CE822F213408F052
:1008F00080E4982F91119CCF922F981B892F3093D1
:10090000E800911103C0203408F4C2CE282FE6CFAE
:0C091000D8DCA8DCA9DCFECFF894FFCFF7
:00000001FF
